 sawindbg

 Timestamp is 6710dd21 (Thu Oct 17 09:47:13 2024)

 Preferred load address is 10000000

 Start         Length     Name                   Class
 0001:00000000 00006480H .text$mn                CODE
 0001:00006480 0000124eH .text$x                 CODE
 0002:00000000 00000104H .CRT$XCA                DATA
 0002:00000104 00000104H .CRT$XCZ                DATA
 0002:00000208 00000104H .CRT$XIA                DATA
 0002:0000030c 00000104H .CRT$XIZ                DATA
 0002:00000410 00000104H .CRT$XPA                DATA
 0002:00000514 00000104H .CRT$XPZ                DATA
 0002:00000618 00000104H .CRT$XTA                DATA
 0002:0000071c 00000104H .CRT$XTZ                DATA
 0002:00000820 00000ba0H .rdata                  DATA
 0002:000013c0 00000180H .rdata$CastGuardVftablesA DATA
 0002:00001540 0000014cH .rdata$CastGuardVftablesC DATA
 0002:0000168c 0000035cH .rdata$r                DATA
 0002:000019e8 00000134H .rdata$sxdata           DATA
 0002:00001b1c 000001e8H .rdata$zzzdbg           DATA
 0002:00001d04 00000104H .rtc$IAA                DATA
 0002:00001e08 00000104H .rtc$IZZ                DATA
 0002:00001f0c 00000104H .rtc$TAA                DATA
 0002:00002010 00000108H .rtc$TZZ                DATA
 0002:00002118 00000598H .xdata$x                DATA
 0002:000026b0 000005a1H .edata                  DATA
 0003:00000000 00000130H .data                   DATA
 0003:00000130 0000017cH .data$r                 DATA
 0003:000002ac 00000194H .data$rs                DATA
 0003:00000440 00000490H .bss                    DATA
 0004:00000000 00000224H .idata$5                DATA
 0004:00000224 0000008cH .idata$2                DATA
 0004:000002b0 00000014H .idata$3                DATA
 0004:000002c4 00000224H .idata$4                DATA
 0004:000004e8 00000642H .idata$6                DATA
 0005:00000000 0000010eH .00cfg                  DATA

  Address         Publics by Value              Rva+Base       Lib:Object

 0000:00000000       ___AbsoluteZero            00000000     <absolute>
 0000:00000000       ___arm64x_extra_rfe_table  00000000     <absolute>
 0000:00000000       ___arm64x_extra_rfe_table_size 00000000     <absolute>
 0000:00000000       ___arm64x_native_entrypoint 00000000     <absolute>
 0000:00000000       ___arm64x_redirection_metadata 00000000     <absolute>
 0000:00000000       ___arm64x_redirection_metadata_count 00000000     <absolute>
 0000:00000000       ___dynamic_value_reloc_table 00000000     <absolute>
 0000:00000000       ___enclave_config          00000000     <absolute>
 0000:00000000       ___guard_check_icall_a64n_fptr 00000000     <absolute>
 0000:00000000       ___guard_eh_cont_count     00000000     <absolute>
 0000:00000000       ___guard_eh_cont_table     00000000     <absolute>
 0000:00000000       ___guard_fids_count        00000000     <absolute>
 0000:00000000       ___guard_fids_table        00000000     <absolute>
 0000:00000000       ___guard_iat_count         00000000     <absolute>
 0000:00000000       ___guard_iat_table         00000000     <absolute>
 0000:00000000       ___guard_longjmp_count     00000000     <absolute>
 0000:00000000       ___guard_longjmp_table     00000000     <absolute>
 0000:00000000       ___hybrid_auxiliary_delayload_iat 00000000     <absolute>
 0000:00000000       ___hybrid_auxiliary_delayload_iat_copy 00000000     <absolute>
 0000:00000000       ___hybrid_auxiliary_iat    00000000     <absolute>
 0000:00000000       ___hybrid_auxiliary_iat_copy 00000000     <absolute>
 0000:00000000       ___hybrid_code_map         00000000     <absolute>
 0000:00000000       ___hybrid_code_map_count   00000000     <absolute>
 0000:00000000       ___hybrid_image_info_bitfield 00000000     <absolute>
 0000:00000000       ___volatile_metadata       00000000     <absolute>
 0000:00000000       ___x64_code_ranges_to_entry_points 00000000     <absolute>
 0000:00000000       ___x64_code_ranges_to_entry_points_count 00000000     <absolute>
 0000:0000000b       ___safe_se_handler_count   0000000b     <absolute>
 0000:00000100       ___guard_flags             00000100     <absolute>
 0000:00000000       ___ImageBase               10000000     <linker-defined>
 0001:00000710       ??0?$AutoArrayPtr@K@@QAE@PAK@Z 10001710 f i sawindbg.obj
 0001:00000720       ??0?$AutoArrayPtr@U_DEBUG_MODULE_PARAMETERS@@@@QAE@PAU_DEBUG_MODULE_PARAMETERS@@@Z 10001720 f i sawindbg.obj
 0001:00000730       ??0?$AutoCOMPtr@UIDebugClient@@@@QAE@PAUIDebugClient@@@Z 10001730 f i sawindbg.obj
 0001:00000740       ??0?$AutoCOMPtr@UIDebugControl@@@@QAE@PAUIDebugControl@@@Z 10001740 f i sawindbg.obj
 0001:00000750       ??0AutoJavaString@@QAE@PAUJNIEnv_@@PAV_jstring@@PBD@Z 10001750 f i sawindbg.obj
 0001:00000770       ??0IDebugOutputCallbacks@@QAE@XZ 10001770 f i sawindbg.obj
 0001:00000780       ??0IUnknown@@QAE@XZ        10001780 f i sawindbg.obj
 0001:00000790       ??0SAOutputCallbacks@@QAE@XZ 10001790 f i sawindbg.obj
 0001:000007b0       ??1?$AutoArrayPtr@K@@QAE@XZ 100017b0 f i sawindbg.obj
 0001:000007c0       ??1?$AutoArrayPtr@U_DEBUG_MODULE_PARAMETERS@@@@QAE@XZ 100017c0 f i sawindbg.obj
 0001:000007d0       ??1?$AutoCOMPtr@UIDebugClient@@@@QAE@XZ 100017d0 f i sawindbg.obj
 0001:00000830       ??1?$AutoCOMPtr@UIDebugControl@@@@QAE@XZ 10001830 f i sawindbg.obj
 0001:00000890       ??1AutoJavaString@@QAE@XZ  10001890 f i sawindbg.obj
 0001:000008f0       ??1SAOutputCallbacks@@QAE@XZ 100018f0 f i sawindbg.obj
 0001:00000920       ??BAutoJavaString@@QAEPBDXZ 10001920 f i sawindbg.obj
 0001:00000930       ??C?$AutoCOMPtr@UIDebugClient@@@@QAEPAUIDebugClient@@XZ 10001930 f i sawindbg.obj
 0001:00000940       ??C?$AutoCOMPtr@UIDebugControl@@@@QAEPAUIDebugControl@@XZ 10001940 f i sawindbg.obj
 0001:00000950       ??_GSAOutputCallbacks@@QAEPAXI@Z 10001950 f i sawindbg.obj
 0001:000009a0       ?AddRef@SAOutputCallbacks@@UAGKXZ 100019a0 f   sawindbg.obj
 0001:000009c0       ?CallObjectMethod@JNIEnv_@@QAAPAV_jobject@@PAV2@PAU_jmethodID@@ZZ 100019c0 f i sawindbg.obj
 0001:000009f0       ?CallVoidMethod@JNIEnv_@@QAAXPAV_jobject@@PAU_jmethodID@@ZZ 100019f0 f i sawindbg.obj
 0001:00000a20       ?ExceptionOccurred@JNIEnv_@@QAEPAV_jthrowable@@XZ 10001a20 f i sawindbg.obj
 0001:00000a30       ?FindClass@JNIEnv_@@QAEPAV_jclass@@PBD@Z 10001a30 f i sawindbg.obj
 0001:00000a50       ?GetByteArrayElements@JNIEnv_@@QAEPACPAV_jbyteArray@@PAE@Z 10001a50 f i sawindbg.obj
 0001:00000a70       ?GetFieldID@JNIEnv_@@QAEPAU_jfieldID@@PAV_jclass@@PBD1@Z 10001a70 f i sawindbg.obj
 0001:00000a90       ?GetLongArrayElements@JNIEnv_@@QAEPA_JPAV_jlongArray@@PAE@Z 10001a90 f i sawindbg.obj
 0001:00000ab0       ?GetLongField@JNIEnv_@@QAE_JPAV_jobject@@PAU_jfieldID@@@Z 10001ab0 f i sawindbg.obj
 0001:00000ad0       ?GetMethodID@JNIEnv_@@QAEPAU_jmethodID@@PAV_jclass@@PBD1@Z 10001ad0 f i sawindbg.obj
 0001:00000af0       ?GetObjectClass@JNIEnv_@@QAEPAV_jclass@@PAV_jobject@@@Z 10001af0 f i sawindbg.obj
 0001:00000b10       ?GetStaticFieldID@JNIEnv_@@QAEPAU_jfieldID@@PAV_jclass@@PBD1@Z 10001b10 f i sawindbg.obj
 0001:00000b30       ?GetStaticObjectField@JNIEnv_@@QAEPAV_jobject@@PAV_jclass@@PAU_jfieldID@@@Z 10001b30 f i sawindbg.obj
 0001:00000b50       ?GetStringUTFChars@JNIEnv_@@QAEPBDPAV_jstring@@PAE@Z 10001b50 f i sawindbg.obj
 0001:00000b70       ?NewByteArray@JNIEnv_@@QAEPAV_jbyteArray@@J@Z 10001b70 f i sawindbg.obj
 0001:00000b90       ?NewLongArray@JNIEnv_@@QAEPAV_jlongArray@@J@Z 10001b90 f i sawindbg.obj
 0001:00000bb0       ?NewStringUTF@JNIEnv_@@QAEPAV_jstring@@PBD@Z 10001bb0 f i sawindbg.obj
 0001:00000bd0       ?Output@SAOutputCallbacks@@UAGJKPBD@Z 10001bd0 f   sawindbg.obj
 0001:00000ce0       ?QueryInterface@SAOutputCallbacks@@UAGJABU_GUID@@PAPAX@Z 10001ce0 f   sawindbg.obj
 0001:00000d80       ?Release@SAOutputCallbacks@@UAGKXZ 10001d80 f   sawindbg.obj
 0001:00000dd0       ?ReleaseByteArrayElements@JNIEnv_@@QAEXPAV_jbyteArray@@PACJ@Z 10001dd0 f i sawindbg.obj
 0001:00000df0       ?ReleaseLongArrayElements@JNIEnv_@@QAEXPAV_jlongArray@@PA_JJ@Z 10001df0 f i sawindbg.obj
 0001:00000e10       ?ReleaseStringUTFChars@JNIEnv_@@QAEXPAV_jstring@@PBD@Z 10001e10 f i sawindbg.obj
 0001:00000e30       ?SetLongField@JNIEnv_@@QAEXPAV_jobject@@PAU_jfieldID@@_J@Z 10001e30 f i sawindbg.obj
 0001:00000e60       ?ThrowNew@JNIEnv_@@QAEJPAV_jclass@@PBD@Z 10001e60 f i sawindbg.obj
 0001:000016d0       ?asPtr@?$AutoArrayPtr@K@@QAEPAKXZ 100026d0 f i sawindbg.obj
 0001:000016e0       ?asPtr@?$AutoArrayPtr@U_DEBUG_MODULE_PARAMETERS@@@@QAEPAU_DEBUG_MODULE_PARAMETERS@@XZ 100026e0 f i sawindbg.obj
 0001:000017e0       ?clearBuffer@SAOutputCallbacks@@QAEXXZ 100027e0 f i sawindbg.obj
 0001:00001810       ?getBuffer@SAOutputCallbacks@@QBEPBDXZ 10002810 f i sawindbg.obj
 0001:00002030       _IsEqualGUID               10003030 f i sawindbg.obj
 0001:00002070       _Java_sun_jvm_hotspot_debugger_windbg_WindbgDebuggerLocal_attach0__I@12 10003070 f   sawindbg.obj
 0001:00002190       _Java_sun_jvm_hotspot_debugger_windbg_WindbgDebuggerLocal_attach0__Ljava_lang_String_2Ljava_lang_String_2@16 10003190 f   sawindbg.obj
 0001:00002430       _Java_sun_jvm_hotspot_debugger_windbg_WindbgDebuggerLocal_consoleExecuteCommand0@12 10003430 f   sawindbg.obj
 0001:00002680       _Java_sun_jvm_hotspot_debugger_windbg_WindbgDebuggerLocal_detach0@8 10003680 f   sawindbg.obj
 0001:000026e0       _Java_sun_jvm_hotspot_debugger_windbg_WindbgDebuggerLocal_getThreadIdFromSysId0@16 100036e0 f   sawindbg.obj
 0001:00002770       _Java_sun_jvm_hotspot_debugger_windbg_WindbgDebuggerLocal_initIDs@8 10003770 f   sawindbg.obj
 0001:00002a30       _Java_sun_jvm_hotspot_debugger_windbg_WindbgDebuggerLocal_lookupByAddress0@16 10003a30 f   sawindbg.obj
 0001:00002b70       _Java_sun_jvm_hotspot_debugger_windbg_WindbgDebuggerLocal_lookupByName0@16 10003b70 f   sawindbg.obj
 0001:00002cc0       _Java_sun_jvm_hotspot_debugger_windbg_WindbgDebuggerLocal_readBytesFromProcess0@24 10003cc0 f   sawindbg.obj
 0001:00002e00       ___local_stdio_printf_options 10003e00 f i sawindbg.obj
 0001:00002e10       __vfprintf_l               10003e10 f i sawindbg.obj
 0001:00002e40       _fprintf                   10003e40 f i sawindbg.obj
 0001:00002e70       _Java_sun_jvm_hotspot_asm_Disassembler_decode@36 10003e70 f   sadis.obj
 0001:00003040       _Java_sun_jvm_hotspot_asm_Disassembler_load_1library@16 10004040 f   sadis.obj
 0001:00003260       __snprintf                 10004260 f i sadis.obj
 0001:000032a0       __vsnprintf                100042a0 f i sadis.obj
 0001:000032e0       __vsnprintf_l              100042e0 f i sadis.obj
 0001:00003608       _DebugCreate@8             10004608 f   dbgeng:dbgeng.dll
 0001:0000360e       ??2@YAPAXI@Z               1000460e f   MSVCRT:new_scalar.obj
 0001:0000364a       ??3@YAXPAXI@Z              1000464a f   MSVCRT:delete_scalar_size.obj
 0001:0000365b       ??_U@YAPAXI@Z              1000465b f   MSVCRT:new_array.obj
 0001:00003666       ??_V@YAXPAX@Z              10004666 f   MSVCRT:delete_array.obj
 0001:0000366b       @__security_check_cookie@4 1000466b f   MSVCRT:secchk.obj
 0001:0000367c       ??1type_info@@UAE@XZ       1000467c f   MSVCRT:std_type_info_static.obj
 0001:00003683       ??_Etype_info@@UAEPAXI@Z   10004683 f i MSVCRT:std_type_info_static.obj
 0001:00003683       ??_Gtype_info@@UAEPAXI@Z   10004683 f i MSVCRT:std_type_info_static.obj
 0001:000036b0       __alloca_probe             100046b0 f   MSVCRT:chkstk.obj
 0001:000036b0       __chkstk                   100046b0 f   MSVCRT:chkstk.obj
 0001:00003af2       __CRT_INIT@12              10004af2 f   MSVCRT:dll_dllmain.obj
 0001:00003afd       __DllMainCRTStartup@12     10004afd f   MSVCRT:dll_dllmain.obj
 0001:00003b28       ??0bad_alloc@std@@AAE@QBD@Z 10004b28 f i MSVCRT:throw_bad_alloc.obj
 0001:00003b4c       ??0bad_alloc@std@@QAE@ABV01@@Z 10004b4c f i MSVCRT:throw_bad_alloc.obj
 0001:00003b6d       ??0bad_alloc@std@@QAE@XZ   10004b6d f i MSVCRT:throw_bad_alloc.obj
 0001:00003b8b       ??0bad_array_new_length@std@@QAE@ABV01@@Z 10004b8b f i MSVCRT:throw_bad_alloc.obj
 0001:00003bac       ??0bad_array_new_length@std@@QAE@XZ 10004bac f i MSVCRT:throw_bad_alloc.obj
 0001:00003bca       ??0exception@std@@QAE@ABV01@@Z 10004bca f i MSVCRT:throw_bad_alloc.obj
 0001:00003c01       ??0exception@std@@QAE@QBDH@Z 10004c01 f i MSVCRT:throw_bad_alloc.obj
 0001:00003c25       ??1bad_alloc@std@@UAE@XZ   10004c25 f i MSVCRT:throw_bad_alloc.obj
 0001:00003c3a       ??1bad_array_new_length@std@@UAE@XZ 10004c3a f i MSVCRT:throw_bad_alloc.obj
 0001:00003c4f       ??1exception@std@@UAE@XZ   10004c4f f i MSVCRT:throw_bad_alloc.obj
 0001:00003c64       ??_Ebad_alloc@std@@UAEPAXI@Z 10004c64 f i MSVCRT:throw_bad_alloc.obj
 0001:00003c64       ??_Gbad_alloc@std@@UAEPAXI@Z 10004c64 f i MSVCRT:throw_bad_alloc.obj
 0001:00003c9c       ??_Ebad_array_new_length@std@@UAEPAXI@Z 10004c9c f i MSVCRT:throw_bad_alloc.obj
 0001:00003c9c       ??_Gbad_array_new_length@std@@UAEPAXI@Z 10004c9c f i MSVCRT:throw_bad_alloc.obj
 0001:00003cd4       ??_Eexception@std@@UAEPAXI@Z 10004cd4 f i MSVCRT:throw_bad_alloc.obj
 0001:00003cd4       ??_Gexception@std@@UAEPAXI@Z 10004cd4 f i MSVCRT:throw_bad_alloc.obj
 0001:00003d0c       ?__scrt_throw_std_bad_alloc@@YAXXZ 10004d0c f   MSVCRT:throw_bad_alloc.obj
 0001:00003d30       ?__scrt_throw_std_bad_array_new_length@@YAXXZ 10004d30 f   MSVCRT:throw_bad_alloc.obj
 0001:00003d54       ?what@exception@std@@UBEPBDXZ 10004d54 f i MSVCRT:throw_bad_alloc.obj
 0001:00003d64       ??3@YAXPAX@Z               10004d64 f   MSVCRT:delete_scalar.obj
 0001:00003d69       ___raise_securityfailure   10004d69 f   MSVCRT:gs_report.obj
 0001:00003d9b       ___report_gsfailure        10004d9b f   MSVCRT:gs_report.obj
 0001:00003ed3       ___report_rangecheckfailure 10004ed3 f   MSVCRT:gs_report.obj
 0001:00003ee2       ___report_securityfailure  10004ee2 f   MSVCRT:gs_report.obj
 0001:00003fe4       ___report_securityfailureEx 10004fe4 f   MSVCRT:gs_report.obj
 0001:0000419e       ___security_init_cookie    1000519e f   MSVCRT:gs_support.obj
 0001:000041fb       _DllMain@12                100051fb f   MSVCRT:dll_dllmain_stub.obj
 0001:00004225       ?__scrt_initialize_type_info@@YAXXZ 10005225 f   MSVCRT:tncleanup.obj
 0001:00004234       ?__scrt_uninitialize_type_info@@YAXXZ 10005234 f   MSVCRT:tncleanup.obj
 0001:00004243       ___local_stdio_scanf_options 10005243 f i MSVCRT:default_local_stdio_options.obj
 0001:00004249       ___scrt_initialize_default_local_stdio_options 10005249 f   MSVCRT:default_local_stdio_options.obj
 0001:0000426d       ?configure_argv@__scrt_narrow_argv_policy@@SAHXZ 1000526d f i MSVCRT:utility.obj
 0001:000042d2       ?initialize_environment@__scrt_narrow_environment_policy@@SAHXZ 100052d2 f i MSVCRT:utility.obj
 0001:00004316       _NtCurrentTeb              10005316 f i MSVCRT:utility.obj
 0001:0000431d       ___scrt_acquire_startup_lock 1000531d f   MSVCRT:utility.obj
 0001:0000435b       ___scrt_dllmain_after_initialize_c 1000535b f   MSVCRT:utility.obj
 0001:00004390       ___scrt_dllmain_before_initialize_c 10005390 f   MSVCRT:utility.obj
 0001:000043a1       ___scrt_dllmain_crt_thread_attach 100053a1 f   MSVCRT:utility.obj
 0001:000043c7       ___scrt_dllmain_crt_thread_detach 100053c7 f   MSVCRT:utility.obj
 0001:000043d7       ___scrt_dllmain_exception_filter 100053d7 f   MSVCRT:utility.obj
 0001:00004418       ___scrt_dllmain_uninitialize_c 10005418 f   MSVCRT:utility.obj
 0001:00004443       ___scrt_dllmain_uninitialize_critical 10005443 f   MSVCRT:utility.obj
 0001:00004453       ___scrt_initialize_crt     10005453 f   MSVCRT:utility.obj
 0001:0000449a       ___scrt_initialize_onexit_tables 1000549a f   MSVCRT:utility.obj
 0001:00004542       ___scrt_is_nonwritable_in_current_image 10005542 f   MSVCRT:utility.obj
 0001:000045fb       ___scrt_release_startup_lock 100055fb f   MSVCRT:utility.obj
 0001:0000461f       ___scrt_uninitialize_crt   1000561f f   MSVCRT:utility.obj
 0001:00004651       __onexit                   10005651 f   MSVCRT:utility.obj
 0001:00004689       _at_quick_exit             10005689 f   MSVCRT:utility.obj
 0001:000046b4       _atexit                    100056b4 f   MSVCRT:utility.obj
 0001:000046ce       ___scrt_get_dyn_tls_init_callback 100056ce f   MSVCRT:dyn_tls_init.obj
 0001:000046d4       ___scrt_fastfail           100056d4 f   MSVCRT:utility_desktop.obj
 0001:00004835       ___scrt_get_show_window_mode 10005835 f   MSVCRT:utility_desktop.obj
 0001:00004872       ___scrt_initialize_mta     10005872 f   MSVCRT:utility_desktop.obj
 0001:00004877       ___scrt_initialize_winrt   10005877 f   MSVCRT:utility_desktop.obj
 0001:0000487a       ___scrt_is_managed_app     1000587a f   MSVCRT:utility_desktop.obj
 0001:000048cc       ___scrt_set_unhandled_exception_filter 100058cc f   MSVCRT:utility_desktop.obj
 0001:000048db       ___scrt_exe_initialize_mta 100058db f   MSVCRT:utility_desktop.obj
 0001:000048db       ___scrt_stub_for_initialize_mta 100058db f   MSVCRT:utility_desktop.obj
 0001:000048de       ___scrt_unhandled_exception_filter@4 100058de f   MSVCRT:utility_desktop.obj
 0001:00004949       __crt_debugger_hook        10005949 f   MSVCRT:utility_desktop.obj
 0001:00004953       __RTC_Initialize           10005953 f   MSVCRT:initsect.obj
 0001:0000498a       __RTC_Terminate            1000598a f   MSVCRT:initsect.obj
 0001:000049d0       __SEH_prolog4              100059d0 f   MSVCRT:sehprolg4.obj
 0001:00004a30       __SEH_epilog4              10005a30 f   MSVCRT:sehprolg4.obj
 0001:00004a49       __except_handler4          10005a49 f   MSVCRT:chandler4gs.obj
 0001:00004a83       @_guard_check_icall_nop@4  10005a83 f i MSVCRT:guard_support.obj
 0001:00004a86       _ReadNoFence               10005a86 f i MSVCRT:guard_support.obj
 0001:00004a92       _ReadPointerNoFence        10005a92 f i MSVCRT:guard_support.obj
 0001:00004a9e       __InlineInterlockedExchangePointer 10005a9e f i MSVCRT:guard_support.obj
 0001:00004aae       ___castguard_check_failure_debugbreak 10005aae f i MSVCRT:guard_support.obj
 0001:00004acf       ___castguard_check_failure_fastfail 10005acf f i MSVCRT:guard_support.obj
 0001:00004af5       ___castguard_check_failure_nop 10005af5 f i MSVCRT:guard_support.obj
 0001:00004af8       ___castguard_check_failure_os_handled 10005af8 f i MSVCRT:guard_support.obj
 0001:00004b48       ___castguard_check_failure_user_handled 10005b48 f i MSVCRT:guard_support.obj
 0001:00004bd0       ___castguard_set_user_handler 10005bd0 f i MSVCRT:guard_support.obj
 0001:00004be2       ___castguard_slow_path_check_debugbreak 10005be2 f i MSVCRT:guard_support.obj
 0001:00004c1a       ___castguard_slow_path_check_fastfail 10005c1a f i MSVCRT:guard_support.obj
 0001:00004c57       ___castguard_slow_path_check_nop 10005c57 f i MSVCRT:guard_support.obj
 0001:00004c5a       ___castguard_slow_path_check_os_handled 10005c5a f i MSVCRT:guard_support.obj
 0001:00004cab       ___castguard_slow_path_check_user_handled 10005cab f i MSVCRT:guard_support.obj
 0001:00004d23       __guard_icall_checks_enforced 10005d23 f i MSVCRT:guard_support.obj
 0001:00004d39       ___isa_available_init      10005d39 f   MSVCRT:cpu_disp.obj
 0001:00004f82       __get_startup_argv_mode    10005f82 f   MSVCRT:argv_mode.obj
 0001:00004f86       ___scrt_is_ucrt_dll_in_use 10005f86 f   MSVCRT:ucrt_detection.obj
 0001:00004f95       _GetLastError@0            10005f95 f   kernel32:KERNEL32.dll
 0001:00004f9b       _GetProcAddress@8          10005f9b f   kernel32:KERNEL32.dll
 0001:00004fa1       _LoadLibraryA@4            10005fa1 f   kernel32:KERNEL32.dll
 0001:00004fa7       _FormatMessageA@28         10005fa7 f   kernel32:KERNEL32.dll
 0001:00004fad       _UnhandledExceptionFilter@4 10005fad f   kernel32:KERNEL32.dll
 0001:00004fb3       _SetUnhandledExceptionFilter@4 10005fb3 f   kernel32:KERNEL32.dll
 0001:00004fb9       _GetCurrentProcess@0       10005fb9 f   kernel32:KERNEL32.dll
 0001:00004fbf       _TerminateProcess@8        10005fbf f   kernel32:KERNEL32.dll
 0001:00004fc5       _IsProcessorFeaturePresent@4 10005fc5 f   kernel32:KERNEL32.dll
 0001:00004fcb       _QueryPerformanceCounter@4 10005fcb f   kernel32:KERNEL32.dll
 0001:00004fd1       _GetCurrentProcessId@0     10005fd1 f   kernel32:KERNEL32.dll
 0001:00004fd7       _GetCurrentThreadId@0      10005fd7 f   kernel32:KERNEL32.dll
 0001:00004fdd       _GetSystemTimeAsFileTime@4 10005fdd f   kernel32:KERNEL32.dll
 0001:00004fe3       _DisableThreadLibraryCalls@4 10005fe3 f   kernel32:KERNEL32.dll
 0001:00004fe9       _InitializeSListHead@4     10005fe9 f   kernel32:KERNEL32.dll
 0001:00004fef       _IsDebuggerPresent@0       10005fef f   kernel32:KERNEL32.dll
 0001:00004ff5       _GetStartupInfoW@4         10005ff5 f   kernel32:KERNEL32.dll
 0001:00004ffb       _GetModuleHandleW@4        10005ffb f   kernel32:KERNEL32.dll
 0001:00005001       ___std_terminate           10006001 f   vcruntime:VCRUNTIME140.dll
 0001:00005007       _strstr                    10006007 f   vcruntime:VCRUNTIME140.dll
 0001:0000500d       ___CxxFrameHandler3        1000600d f   vcruntime:VCRUNTIME140.dll
 0001:00005013       _memset                    10006013 f   vcruntime:VCRUNTIME140.dll
 0001:00005019       _strchr                    10006019 f   vcruntime:VCRUNTIME140.dll
 0001:0000501f       ___std_exception_copy      1000601f f   vcruntime:VCRUNTIME140.dll
 0001:00005025       ___std_exception_destroy   10006025 f   vcruntime:VCRUNTIME140.dll
 0001:0000502b       __CxxThrowException@8      1000602b f   vcruntime:VCRUNTIME140.dll
 0001:00005031       ___std_type_info_destroy_list 10006031 f   vcruntime:VCRUNTIME140.dll
 0001:00005037       ___current_exception       10006037 f   vcruntime:VCRUNTIME140.dll
 0001:0000503d       ___current_exception_context 1000603d f   vcruntime:VCRUNTIME140.dll
 0001:00005043       __except_handler4_common   10006043 f   vcruntime:VCRUNTIME140.dll
 0001:00005049       ___acrt_iob_func           10006049 f   ucrt:api-ms-win-crt-stdio-l1-1-0.dll
 0001:0000504f       ___stdio_common_vfprintf   1000604f f   ucrt:api-ms-win-crt-stdio-l1-1-0.dll
 0001:00005055       _free                      10006055 f   ucrt:api-ms-win-crt-heap-l1-1-0.dll
 0001:0000505b       _malloc                    1000605b f   ucrt:api-ms-win-crt-heap-l1-1-0.dll
 0001:00005061       _realloc                   10006061 f   ucrt:api-ms-win-crt-heap-l1-1-0.dll
 0001:00005067       ___stdio_common_vsprintf   10006067 f   ucrt:api-ms-win-crt-stdio-l1-1-0.dll
 0001:0000506d       __errno                    1000606d f   ucrt:api-ms-win-crt-runtime-l1-1-0.dll
 0001:00005073       _strerror                  10006073 f   ucrt:api-ms-win-crt-runtime-l1-1-0.dll
 0001:00005079       _strncpy                   10006079 f   ucrt:api-ms-win-crt-string-l1-1-0.dll
 0001:0000507f       __callnewh                 1000607f f   ucrt:api-ms-win-crt-heap-l1-1-0.dll
 0001:00005085       __initterm                 10006085 f   ucrt:api-ms-win-crt-runtime-l1-1-0.dll
 0001:0000508b       __initterm_e               1000608b f   ucrt:api-ms-win-crt-runtime-l1-1-0.dll
 0001:00005091       __seh_filter_dll           10006091 f   ucrt:api-ms-win-crt-runtime-l1-1-0.dll
 0001:00005097       __configure_narrow_argv    10006097 f   ucrt:api-ms-win-crt-runtime-l1-1-0.dll
 0001:0000509d       __initialize_narrow_environment 1000609d f   ucrt:api-ms-win-crt-runtime-l1-1-0.dll
 0001:000050a3       __initialize_onexit_table  100060a3 f   ucrt:api-ms-win-crt-runtime-l1-1-0.dll
 0001:000050a9       __register_onexit_function 100060a9 f   ucrt:api-ms-win-crt-runtime-l1-1-0.dll
 0001:000050af       __execute_onexit_table     100060af f   ucrt:api-ms-win-crt-runtime-l1-1-0.dll
 0001:000050b5       __crt_atexit               100060b5 f   ucrt:api-ms-win-crt-runtime-l1-1-0.dll
 0001:000050bb       __crt_at_quick_exit        100060bb f   ucrt:api-ms-win-crt-runtime-l1-1-0.dll
 0001:000050c1       __cexit                    100060c1 f   ucrt:api-ms-win-crt-runtime-l1-1-0.dll
 0001:000050c7       _terminate                 100060c7 f   ucrt:api-ms-win-crt-runtime-l1-1-0.dll
 0001:000050cd       ___acrt_initialize         100060cd f   MSVCRT:ucrt_stubs.obj
 0001:000050cd       ___scrt_stub_for_acrt_initialize 100060cd f   MSVCRT:ucrt_stubs.obj
 0001:000050cd       ___vcrt_initialize         100060cd f   MSVCRT:ucrt_stubs.obj
 0001:000050d0       ___acrt_thread_attach      100060d0 f   MSVCRT:ucrt_stubs.obj
 0001:000050d0       ___scrt_stub_for_acrt_thread_attach 100060d0 f   MSVCRT:ucrt_stubs.obj
 0001:000050d0       ___vcrt_thread_attach      100060d0 f   MSVCRT:ucrt_stubs.obj
 0001:000050d3       ___acrt_thread_detach      100060d3 f   MSVCRT:ucrt_stubs.obj
 0001:000050d3       ___scrt_stub_for_acrt_thread_detach 100060d3 f   MSVCRT:ucrt_stubs.obj
 0001:000050d3       ___vcrt_thread_detach      100060d3 f   MSVCRT:ucrt_stubs.obj
 0001:000050d6       ___acrt_uninitialize       100060d6 f   MSVCRT:ucrt_stubs.obj
 0001:000050d6       ___scrt_stub_for_acrt_uninitialize 100060d6 f   MSVCRT:ucrt_stubs.obj
 0001:000050d6       ___vcrt_uninitialize       100060d6 f   MSVCRT:ucrt_stubs.obj
 0001:000050d9       ___acrt_uninitialize_critical 100060d9 f   MSVCRT:ucrt_stubs.obj
 0001:000050d9       ___scrt_stub_for_acrt_uninitialize_critical 100060d9 f   MSVCRT:ucrt_stubs.obj
 0001:000050d9       ___vcrt_uninitialize_critical 100060d9 f   MSVCRT:ucrt_stubs.obj
 0001:000050dc       ___scrt_stub_for_is_c_termination_complete 100060dc f   MSVCRT:ucrt_stubs.obj
 0001:000050dc       __is_c_termination_complete 100060dc f   MSVCRT:ucrt_stubs.obj
 0001:000050df       __filter_x86_sse2_floating_point_exception 100060df f   MSVCRT:x86_exception_filter.obj
 0001:000050df       __filter_x86_sse2_floating_point_exception_default 100060df f   MSVCRT:x86_exception_filter.obj
 0002:00000000       ___xc_a                    10009000     MSVCRT:initializers.obj
 0002:00000104       ___xc_z                    10009104     MSVCRT:initializers.obj
 0002:00000208       ___xi_a                    10009208     MSVCRT:initializers.obj
 0002:0000030c       ___xi_z                    1000930c     MSVCRT:initializers.obj
 0002:00000410       ___xp_a                    10009410     MSVCRT:initializers.obj
 0002:00000514       ___xp_z                    10009514     MSVCRT:initializers.obj
 0002:00000618       ___xt_a                    10009618     MSVCRT:initializers.obj
 0002:0000071c       ___xt_z                    1000971c     MSVCRT:initializers.obj
 0002:00000820       ??_C@_0CL@BJCJOPKP@sun?1jvm?1hotspot?1debugger?1Debugg@ 10009820     sawindbg.obj
 0002:00000854       ??_C@_0BD@JFADHEFE@Ljava?1lang?1String?$DL@ 10009854     sawindbg.obj
 0002:0000086c       ??_C@_09NDJHOMOJ@imagePath@ 1000986c     sawindbg.obj
 0002:00000878       ??_C@_0L@IBJLJICF@symbolPath@ 10009878     sawindbg.obj
 0002:00000888       ??_C@_01LELAEKIP@J@        10009888     sawindbg.obj
 0002:0000088c       ??_C@_0BA@ENOAPBEH@ptrIDebugClient@ 1000988c     sawindbg.obj
 0002:000008a0       ??_C@_0BB@FKGMCAMI@ptrIDebugControl@ 100098a0     sawindbg.obj
 0002:000008b4       ??_C@_0BE@HEDMCBCH@ptrIDebugDataSpaces@ 100098b4     sawindbg.obj
 0002:000008cc       ??_C@_0BJ@NECGJCMP@ptrIDebugOutputCallbacks@ 100098cc     sawindbg.obj
 0002:000008ec       ??_C@_0BC@NFADOE@ptrIDebugAdvanced@ 100098ec     sawindbg.obj
 0002:00000904       ??_C@_0BB@CGICJHBO@ptrIDebugSymbols@ 10009904     sawindbg.obj
 0002:00000918       ??_C@_0BH@MKNGBFEC@ptrIDebugSystemObjects@ 10009918     sawindbg.obj
 0002:00000934       ??_C@_0BI@HMPCDPNN@?$CILjava?1lang?1String?$DLJJ?$CJV@ 10009934     sawindbg.obj
 0002:00000950       ??_C@_0O@BAEIOKDM@addLoadObject@ 10009950     sawindbg.obj
 0002:00000960       ??_C@_04OHLIFDMD@?$CIJ?$CJV@ 10009960     sawindbg.obj
 0002:00000968       ??_C@_09IDCNHNJH@addThread@ 10009968     sawindbg.obj
 0002:00000978       ??_C@_0ED@MJCAPJHB@?$CILjava?1lang?1String?$DLJ?$CJLsun?1jvm?1h@ 10009978     sawindbg.obj
 0002:000009c8       ??_C@_0BE@PHFCBNMF@createClosestSymbol@ 100099c8     sawindbg.obj
 0002:000009e0       ??_C@_06FABFLPEO@?$CIJ?$FLJ?$CJV@ 100099e0     sawindbg.obj
 0002:000009e8       ??_C@_0BM@LHHFOJLN@setThreadIntegerRegisterSet@ 100099e8     sawindbg.obj
 0002:00000a10       ??_7SAOutputCallbacks@@6B@ 10009a10     sawindbg.obj
 0002:00000a24       __GUID_00000000_0000_0000_c000_000000000046 10009a24     sawindbg.obj
 0002:00000a38       __GUID_4bf58045_d654_4c40_b0af_683090f356dc 10009a38     sawindbg.obj
 0002:00000a4c       ??_C@_0CA@CHBBHPBL@out?5of?5memory?5debugger?5output?$CB?6@ 10009a4c     sawindbg.obj
 0002:00000a74       __GUID_27fe5639_8407_4f47_8364_ee118fb08ac8 10009a74     sawindbg.obj
 0002:00000a88       __GUID_5182e668_105e_416e_ad92_24ef800424ba 10009a88     sawindbg.obj
 0002:00000a9c       __GUID_88f7dfab_3ea7_4c3a_aefb_c4e8106173aa 10009a9c     sawindbg.obj
 0002:00000ab0       __GUID_f2df5f53_071f_47bd_9de6_5734c3fed689 10009ab0     sawindbg.obj
 0002:00000ac4       __GUID_8c31e98c_983a_48a5_9016_6fe5d667a950 10009ac4     sawindbg.obj
 0002:00000ad8       __GUID_6b86fe2c_2c4f_4f0c_9da2_174311acc327 10009ad8     sawindbg.obj
 0002:00000aec       ??_C@_0DG@KFKFAAAK@Windbg?5Error?3?5not?5able?5to?5creat@ 10009aec     sawindbg.obj
 0002:00000b2c       ??_C@_0CM@HMPHNLCI@Windbg?5Error?3?5not?5able?5to?5get?5I@ 10009b2c     sawindbg.obj
 0002:00000b60       ??_C@_0DH@MEIJIPLO@Windbg?5Error?3?5not?5able?5to?5get?5I@ 10009b60     sawindbg.obj
 0002:00000ba4       ??_C@_0DF@EJNGMFHL@Windbg?5Error?3?5not?5able?5to?5get?5I@ 10009ba4     sawindbg.obj
 0002:00000be4       ??_C@_0DE@BLHEEHEB@Windbg?5Error?3?5not?5able?5to?5get?5I@ 10009be4     sawindbg.obj
 0002:00000c24       ??_C@_0DK@CBFLKIDH@Windbg?5Error?3?5not?5able?5to?5get?5I@ 10009c24     sawindbg.obj
 0002:00000c6c       ??_C@_0CD@LLBBNFEA@Windbg?5Error?3?5OpenDumpFile?5fail@ 10009c6c     sawindbg.obj
 0002:00000c98       ??_C@_0CD@OHANEGIO@Windbg?5Error?3?5WaitForEvent?5fail@ 10009c98     sawindbg.obj
 0002:00000cc4       ??_C@_0CE@NLOIALLD@Windbg?5Error?3?5AttachProcess?5fai@ 10009cc4     sawindbg.obj
 0002:00000cf0       ??_C@_0CH@OOOMOIHO@Windbg?5Error?3?5GetNumberModules?5@ 10009cf0     sawindbg.obj
 0002:00000d20       ??_C@_0CP@GGPCODCJ@out?5of?5memory?5to?5allocate?5debug@ 10009d20     sawindbg.obj
 0002:00000d58       ??_C@_0CK@OGHLJMOC@Windbg?5Error?3?5GetModuleParamete@ 10009d58     sawindbg.obj
 0002:00000d8c       ??_C@_0CF@IPJIKFLG@Windbg?5Error?3?5GetModuleNames?5fa@ 10009d8c     sawindbg.obj
 0002:00000db8       ??_C@_0CH@DLOHNIAK@Windbg?5Error?3?5GetNumberThreads?5@ 10009db8     sawindbg.obj
 0002:00000de8       ??_C@_0CG@KABLKJNP@out?5of?5memory?5to?5allocate?5threa@ 10009de8     sawindbg.obj
 0002:00000e18       ??_C@_0CK@FNPIPCCJ@Windbg?5Error?3?5GetThreadIdsByInd@ 10009e18     sawindbg.obj
 0002:00000e4c       ??_C@_0CH@DDGKENOM@Windbg?5Error?3?5SetCurrentThread?5@ 10009e4c     sawindbg.obj
 0002:00000e7c       ??_C@_0CP@GPDFIPCF@Windbg?5Error?3?5GetCurrentThreadS@ 10009e7c     sawindbg.obj
 0002:00000eb4       ??_C@_0CC@DGPMKKCL@Windbg?5Error?3?5ReadVirtual?5faile@ 10009eb4     sawindbg.obj
 0002:00000edc       ??_C@_0CM@BCOGMGMH@Windbg?5Error?3?5GetThreadIdBySyst@ 10009edc     sawindbg.obj
 0002:00000f10       ??_C@_0CD@EHILJEIM@Windbg?5Error?3?5CreateClient?5fail@ 10009f10     sawindbg.obj
 0002:00000f3c       ??_C@_0DE@HJKLOPIF@Windbg?5Error?3?5QueryInterface?5?$CII@ 10009f3c     sawindbg.obj
 0002:00000f7c       ??_C@_0CJ@LPJOGDLF@Windbg?5Error?3?5SetOutputCallback@ 10009f7c     sawindbg.obj
 0002:00000fad       ??_C@_00CNPNBAHC@@         10009fad     sawindbg.obj
 0002:00000fb0       ??_C@_02MOLJINC@?3?3@      10009fb0     sawindbg.obj
 0002:00000fb4       ??_C@_04HDOCAJNK@?$CFs?$CFs@ 10009fb4     sadis.obj
 0002:00000fbc       ??_C@_0BM@DBCALOPO@decode_instructions_virtual@ 10009fbc     sadis.obj
 0002:00000fe0       ??_C@_0DP@IEGOKKOO@?$CILsun?1jvm?1hotspot?1asm?1Instructi@ 10009fe0     sadis.obj
 0002:0000102c       ??_C@_0M@IHKAILBK@handleEvent@ 1000a02c     sadis.obj
 0002:0000103c       ??_C@_0DO@KENEIINN@?$CILsun?1jvm?1hotspot?1asm?1Instructi@ 1000a03c     sadis.obj
 0002:00001088       ??_C@_08DCIFBHIL@rawPrint@ 1000a088     sadis.obj
 0002:00001098       ??_7type_info@@6B@         1000a098     MSVCRT:std_type_info_static.obj
 0002:000010a0       __pDefaultRawDllMain       1000a0a0     MSVCRT:dll_dllmain.obj
 0002:000010a0       __pRawDllMain              1000a0a0     MSVCRT:dll_dllmain.obj
 0002:000010a8       ??_7exception@std@@6B@     1000a0a8     MSVCRT:throw_bad_alloc.obj
 0002:000010b4       ??_C@_0BC@EOODALEL@Unknown?5exception@ 1000a0b4     MSVCRT:throw_bad_alloc.obj
 0002:000010d0       ??_7bad_alloc@std@@6B@     1000a0d0     MSVCRT:throw_bad_alloc.obj
 0002:000010dc       ??_C@_0P@GHFPNOJB@bad?5allocation@ 1000a0dc     MSVCRT:throw_bad_alloc.obj
 0002:000010f4       ??_7bad_array_new_length@std@@6B@ 1000a0f4     MSVCRT:throw_bad_alloc.obj
 0002:00001100       ??_C@_0BF@KINCDENJ@bad?5array?5new?5length@ 1000a100     MSVCRT:throw_bad_alloc.obj
 0002:00001128       __load_config_used         1000a128     MSVCRT:loadcfg.obj
 0002:000013c0       ___CastGuardVftablesStart  1000a3c0     MSVCRT:guard_support.obj
 0002:00001540       ___CastGuardVftablesEnd    1000a540     MSVCRT:guard_support.obj
 0002:0000168c       ??_R3IUnknown@@8           1000a68c     sawindbg.obj
 0002:000016a0       ??_R2IUnknown@@8           1000a6a0     sawindbg.obj
 0002:000016a8       ??_R1A@?0A@EA@IUnknown@@8  1000a6a8     sawindbg.obj
 0002:000016cc       ??_R3IDebugOutputCallbacks@@8 1000a6cc     sawindbg.obj
 0002:000016e0       ??_R2IDebugOutputCallbacks@@8 1000a6e0     sawindbg.obj
 0002:000016ec       ??_R1A@?0A@EA@IDebugOutputCallbacks@@8 1000a6ec     sawindbg.obj
 0002:00001710       ??_R4SAOutputCallbacks@@6B@ 1000a710     sawindbg.obj
 0002:00001728       ??_R3SAOutputCallbacks@@8  1000a728     sawindbg.obj
 0002:0000173c       ??_R2SAOutputCallbacks@@8  1000a73c     sawindbg.obj
 0002:0000174c       ??_R1A@?0A@EA@SAOutputCallbacks@@8 1000a74c     sawindbg.obj
 0002:00001770       ??_R4type_info@@6B@        1000a770     MSVCRT:std_type_info_static.obj
 0002:00001788       ??_R3type_info@@8          1000a788     MSVCRT:std_type_info_static.obj
 0002:0000179c       ??_R2type_info@@8          1000a79c     MSVCRT:std_type_info_static.obj
 0002:000017a4       ??_R1A@?0A@EA@type_info@@8 1000a7a4     MSVCRT:std_type_info_static.obj
 0002:000017c8       ??_R4exception@std@@6B@    1000a7c8     MSVCRT:throw_bad_alloc.obj
 0002:000017e0       ??_R3exception@std@@8      1000a7e0     MSVCRT:throw_bad_alloc.obj
 0002:000017f4       ??_R2exception@std@@8      1000a7f4     MSVCRT:throw_bad_alloc.obj
 0002:000017fc       ??_R1A@?0A@EA@exception@std@@8 1000a7fc     MSVCRT:throw_bad_alloc.obj
 0002:00001820       ??_R4bad_alloc@std@@6B@    1000a820     MSVCRT:throw_bad_alloc.obj
 0002:00001838       ??_R3bad_alloc@std@@8      1000a838     MSVCRT:throw_bad_alloc.obj
 0002:0000184c       ??_R2bad_alloc@std@@8      1000a84c     MSVCRT:throw_bad_alloc.obj
 0002:00001858       ??_R1A@?0A@EA@bad_alloc@std@@8 1000a858     MSVCRT:throw_bad_alloc.obj
 0002:0000187c       ??_R4bad_array_new_length@std@@6B@ 1000a87c     MSVCRT:throw_bad_alloc.obj
 0002:00001894       ??_R3bad_array_new_length@std@@8 1000a894     MSVCRT:throw_bad_alloc.obj
 0002:000018a8       ??_R2bad_array_new_length@std@@8 1000a8a8     MSVCRT:throw_bad_alloc.obj
 0002:000018b8       ??_R1A@?0A@EA@bad_array_new_length@std@@8 1000a8b8     MSVCRT:throw_bad_alloc.obj
 0002:000019e8       ___safe_se_handler_table   1000a9e8     <linker-defined>
 0002:00001d04       ___rtc_iaa                 1000ad04     MSVCRT:initsect.obj
 0002:00001e08       ___rtc_izz                 1000ae08     MSVCRT:initsect.obj
 0002:00001f0c       ___rtc_taa                 1000af0c     MSVCRT:initsect.obj
 0002:00002010       ___rtc_tzz                 1000b010     MSVCRT:initsect.obj
 0002:00002470       __TI2?AVbad_alloc@std@@    1000b470     MSVCRT:throw_bad_alloc.obj
 0002:00002484       __CTA2?AVbad_alloc@std@@   1000b484     MSVCRT:throw_bad_alloc.obj
 0002:00002494       __CT??_R0?AVbad_alloc@std@@@8??0bad_alloc@std@@QAE@ABV01@@Z12 1000b494     MSVCRT:throw_bad_alloc.obj
 0002:000024b4       __CT??_R0?AVexception@std@@@8??0exception@std@@QAE@ABV01@@Z12 1000b4b4     MSVCRT:throw_bad_alloc.obj
 0002:000024d4       __TI3?AVbad_array_new_length@std@@ 1000b4d4     MSVCRT:throw_bad_alloc.obj
 0002:000024e8       __CTA3?AVbad_array_new_length@std@@ 1000b4e8     MSVCRT:throw_bad_alloc.obj
 0002:000024fc       __CT??_R0?AVbad_array_new_length@std@@@8??0bad_array_new_length@std@@QAE@ABV01@@Z12 1000b4fc     MSVCRT:throw_bad_alloc.obj
 0003:00000000       ___security_cookie_complement 1000c000     MSVCRT:gs_cookie.obj
 0003:00000004       ___security_cookie         1000c004     MSVCRT:gs_cookie.obj
 0003:00000010       ___scrt_native_dllmain_reason 1000c010     MSVCRT:utility.obj
 0003:00000020       ___isa_enabled             1000c020     MSVCRT:cpu_disp.obj
 0003:00000024       ___scrt_ucrt_dll_is_in_use 1000c024     MSVCRT:ucrt_stubs.obj
 0003:00000130       ??_R0?AVbad_alloc@std@@@8  1000c130     MSVCRT:throw_bad_alloc.obj
 0003:00000154       ??_R0?AVexception@std@@@8  1000c154     MSVCRT:throw_bad_alloc.obj
 0003:00000178       ??_R0?AVbad_array_new_length@std@@@8 1000c178     MSVCRT:throw_bad_alloc.obj
 0003:000002ac       ??_R0?AUIUnknown@@@8       1000c2ac     sawindbg.obj
 0003:000002c8       ??_R0?AUIDebugOutputCallbacks@@@8 1000c2c8     sawindbg.obj
 0003:000002f4       ??_R0?AVSAOutputCallbacks@@@8 1000c2f4     sawindbg.obj
 0003:0000031c       ??_R0?AVtype_info@@@8      1000c31c     MSVCRT:std_type_info_static.obj
 0003:00000440       ?_OptionsStorage@?1??__local_stdio_printf_options@@9@4_KA 1000c440     sawindbg.obj
 0003:00000850       ?__type_info_root_node@@3U__type_info_node@@A 1000c850     MSVCRT:tncleanup.obj
 0003:00000860       ?_OptionsStorage@?1??__local_stdio_scanf_options@@9@4_KA 1000c860     MSVCRT:default_local_stdio_options.obj
 0003:0000086c       ___scrt_current_native_startup_state 1000c86c     MSVCRT:utility.obj
 0003:00000870       ___scrt_native_startup_lock 1000c870     MSVCRT:utility.obj
 0003:00000898       ___scrt_debugger_hook_flag 1000c898     MSVCRT:utility_desktop.obj
 0003:0000089c       ___castguard_check_failure_user_handled_fptr 1000c89c     MSVCRT:guard_support.obj
 0003:000008a0       ___isa_available           1000c8a0     MSVCRT:cpu_disp.obj
 0003:000008a4       ___favor                   1000c8a4     MSVCRT:cpu_disp.obj
 0003:000008b0       ?_OptionsStorage@?1??__local_stdio_printf_options@@9@9 1000c8b0     <common>
 0003:000008c4       ___dyn_tls_init_callback   1000c8c4     <common>
 0004:00000000       __imp__IsProcessorFeaturePresent@4 1000d000     kernel32:KERNEL32.dll
 0004:00000004       __imp__GetModuleHandleW@4  1000d004     kernel32:KERNEL32.dll
 0004:00000008       __imp__GetLastError@0      1000d008     kernel32:KERNEL32.dll
 0004:0000000c       __imp__GetProcAddress@8    1000d00c     kernel32:KERNEL32.dll
 0004:00000010       __imp__LoadLibraryA@4      1000d010     kernel32:KERNEL32.dll
 0004:00000014       __imp__FormatMessageA@28   1000d014     kernel32:KERNEL32.dll
 0004:00000018       __imp__UnhandledExceptionFilter@4 1000d018     kernel32:KERNEL32.dll
 0004:0000001c       __imp__SetUnhandledExceptionFilter@4 1000d01c     kernel32:KERNEL32.dll
 0004:00000020       __imp__GetCurrentProcess@0 1000d020     kernel32:KERNEL32.dll
 0004:00000024       __imp__TerminateProcess@8  1000d024     kernel32:KERNEL32.dll
 0004:00000028       __imp__IsDebuggerPresent@0 1000d028     kernel32:KERNEL32.dll
 0004:0000002c       __imp__QueryPerformanceCounter@4 1000d02c     kernel32:KERNEL32.dll
 0004:00000030       __imp__GetCurrentProcessId@0 1000d030     kernel32:KERNEL32.dll
 0004:00000034       __imp__GetCurrentThreadId@0 1000d034     kernel32:KERNEL32.dll
 0004:00000038       __imp__GetSystemTimeAsFileTime@4 1000d038     kernel32:KERNEL32.dll
 0004:0000003c       __imp__DisableThreadLibraryCalls@4 1000d03c     kernel32:KERNEL32.dll
 0004:00000040       __imp__InitializeSListHead@4 1000d040     kernel32:KERNEL32.dll
 0004:00000044       __imp__GetStartupInfoW@4   1000d044     kernel32:KERNEL32.dll
 0004:00000048       \177KERNEL32_NULL_THUNK_DATA 1000d048     kernel32:KERNEL32.dll
 0004:00000080       __imp____current_exception 1000d080     vcruntime:VCRUNTIME140.dll
 0004:00000084       __imp___except_handler4_common 1000d084     vcruntime:VCRUNTIME140.dll
 0004:00000088       __imp____std_terminate     1000d088     vcruntime:VCRUNTIME140.dll
 0004:0000008c       __imp__strstr              1000d08c     vcruntime:VCRUNTIME140.dll
 0004:00000090       __imp____CxxFrameHandler3  1000d090     vcruntime:VCRUNTIME140.dll
 0004:00000094       __imp__memset              1000d094     vcruntime:VCRUNTIME140.dll
 0004:00000098       __imp__strchr              1000d098     vcruntime:VCRUNTIME140.dll
 0004:0000009c       __imp____std_exception_copy 1000d09c     vcruntime:VCRUNTIME140.dll
 0004:000000a0       __imp____std_exception_destroy 1000d0a0     vcruntime:VCRUNTIME140.dll
 0004:000000a4       __imp___CxxThrowException@8 1000d0a4     vcruntime:VCRUNTIME140.dll
 0004:000000a8       __imp____std_type_info_destroy_list 1000d0a8     vcruntime:VCRUNTIME140.dll
 0004:000000ac       __imp____current_exception_context 1000d0ac     vcruntime:VCRUNTIME140.dll
 0004:000000b0       \177VCRUNTIME140_NULL_THUNK_DATA 1000d0b0     vcruntime:VCRUNTIME140.dll
 0004:000000e4       __imp__realloc             1000d0e4     ucrt:api-ms-win-crt-heap-l1-1-0.dll
 0004:000000e8       __imp__malloc              1000d0e8     ucrt:api-ms-win-crt-heap-l1-1-0.dll
 0004:000000ec       __imp___callnewh           1000d0ec     ucrt:api-ms-win-crt-heap-l1-1-0.dll
 0004:000000f0       __imp__free                1000d0f0     ucrt:api-ms-win-crt-heap-l1-1-0.dll
 0004:000000f4       \177api-ms-win-crt-heap-l1-1-0_NULL_THUNK_DATA 1000d0f4     ucrt:api-ms-win-crt-heap-l1-1-0.dll
 0004:00000120       __imp__terminate           1000d120     ucrt:api-ms-win-crt-runtime-l1-1-0.dll
 0004:00000124       __imp___crt_atexit         1000d124     ucrt:api-ms-win-crt-runtime-l1-1-0.dll
 0004:00000128       __imp___errno              1000d128     ucrt:api-ms-win-crt-runtime-l1-1-0.dll
 0004:0000012c       __imp__strerror            1000d12c     ucrt:api-ms-win-crt-runtime-l1-1-0.dll
 0004:00000130       __imp___execute_onexit_table 1000d130     ucrt:api-ms-win-crt-runtime-l1-1-0.dll
 0004:00000134       __imp___cexit              1000d134     ucrt:api-ms-win-crt-runtime-l1-1-0.dll
 0004:00000138       __imp___crt_at_quick_exit  1000d138     ucrt:api-ms-win-crt-runtime-l1-1-0.dll
 0004:0000013c       __imp___initterm           1000d13c     ucrt:api-ms-win-crt-runtime-l1-1-0.dll
 0004:00000140       __imp___initterm_e         1000d140     ucrt:api-ms-win-crt-runtime-l1-1-0.dll
 0004:00000144       __imp___seh_filter_dll     1000d144     ucrt:api-ms-win-crt-runtime-l1-1-0.dll
 0004:00000148       __imp___configure_narrow_argv 1000d148     ucrt:api-ms-win-crt-runtime-l1-1-0.dll
 0004:0000014c       __imp___initialize_narrow_environment 1000d14c     ucrt:api-ms-win-crt-runtime-l1-1-0.dll
 0004:00000150       __imp___initialize_onexit_table 1000d150     ucrt:api-ms-win-crt-runtime-l1-1-0.dll
 0004:00000154       __imp___register_onexit_function 1000d154     ucrt:api-ms-win-crt-runtime-l1-1-0.dll
 0004:00000158       \177api-ms-win-crt-runtime-l1-1-0_NULL_THUNK_DATA 1000d158     ucrt:api-ms-win-crt-runtime-l1-1-0.dll
 0004:0000018c       __imp____stdio_common_vfprintf 1000d18c     ucrt:api-ms-win-crt-stdio-l1-1-0.dll
 0004:00000190       __imp____acrt_iob_func     1000d190     ucrt:api-ms-win-crt-stdio-l1-1-0.dll
 0004:00000194       __imp____stdio_common_vsprintf 1000d194     ucrt:api-ms-win-crt-stdio-l1-1-0.dll
 0004:00000198       \177api-ms-win-crt-stdio-l1-1-0_NULL_THUNK_DATA 1000d198     ucrt:api-ms-win-crt-stdio-l1-1-0.dll
 0004:000001c4       __imp__strncpy             1000d1c4     ucrt:api-ms-win-crt-string-l1-1-0.dll
 0004:000001c8       \177api-ms-win-crt-string-l1-1-0_NULL_THUNK_DATA 1000d1c8     ucrt:api-ms-win-crt-string-l1-1-0.dll
 0004:000001f4       __imp__DebugCreate@8       1000d1f4     dbgeng:dbgeng.dll
 0004:000001f8       \177dbgeng_NULL_THUNK_DATA 1000d1f8     dbgeng:dbgeng.dll
 0004:00000224       __IMPORT_DESCRIPTOR_dbgeng 1000d224     dbgeng:dbgeng.dll
 0004:00000238       __IMPORT_DESCRIPTOR_KERNEL32 1000d238     kernel32:KERNEL32.dll
 0004:0000024c       __IMPORT_DESCRIPTOR_VCRUNTIME140 1000d24c     vcruntime:VCRUNTIME140.dll
 0004:00000260       __IMPORT_DESCRIPTOR_api-ms-win-crt-stdio-l1-1-0 1000d260     ucrt:api-ms-win-crt-stdio-l1-1-0.dll
 0004:00000274       __IMPORT_DESCRIPTOR_api-ms-win-crt-heap-l1-1-0 1000d274     ucrt:api-ms-win-crt-heap-l1-1-0.dll
 0004:00000288       __IMPORT_DESCRIPTOR_api-ms-win-crt-runtime-l1-1-0 1000d288     ucrt:api-ms-win-crt-runtime-l1-1-0.dll
 0004:0000029c       __IMPORT_DESCRIPTOR_api-ms-win-crt-string-l1-1-0 1000d29c     ucrt:api-ms-win-crt-string-l1-1-0.dll
 0004:000002b0       __NULL_IMPORT_DESCRIPTOR   1000d2b0     dbgeng:dbgeng.dll
 0005:00000000       ___guard_check_icall_fptr  1000e000     MSVCRT:guard_support.obj
 0005:00000004       ___guard_xfg_check_icall_fptr 1000e004     MSVCRT:guard_support.obj
 0005:00000008       ___castguard_check_failure_os_handled_fptr 1000e008     MSVCRT:guard_support.obj

 entry point at        0001:0000032a

 Static symbols

 0000:ffff0000       .debug$S                   10000000     sawindbg.exp
 0000:ffff2000       __guard_fids___except_handler4 10000000     MSVCRT:chandler4gs.obj
 0000:00000000       _volmd                     10000000     MSVCRT:cpu_disp.obj
 0000:ffff2000       __guard_fids_?dllmain_dispatch@@YAHQAUHINSTANCE__@@KQAX@Z 10000000     MSVCRT:dll_dllmain.obj
 0000:00000000       _volmd                     10000000     MSVCRT:gs_report.obj
 0000:ffff2000       __guard_fids__             10000000     MSVCRT:guard_support.obj
 0000:ffff2000       __guard_fids__             10000000     MSVCRT:guard_support.obj
 0000:ffff2000       __guard_fids___guard_icall_checks_enforced 10000000     MSVCRT:guard_support.obj
 0000:00000000       _volmd                     10000000     MSVCRT:guard_support.obj
 0000:00000000       _volmd                     10000000     MSVCRT:guard_support.obj
 0000:00000000       _volmd                     10000000     MSVCRT:guard_support.obj
 0000:00000000       _volmd                     10000000     MSVCRT:guard_support.obj
 0000:00000000       _volmd                     10000000     MSVCRT:guard_support.obj
 0000:00000000       _volmd                     10000000     MSVCRT:guard_support.obj
 0000:00000000       _volmd                     10000000     MSVCRT:guard_support.obj
 0000:00000000       _volmd                     10000000     MSVCRT:guard_support.obj
 0000:00000000       _volmd                     10000000     MSVCRT:guard_support.obj
 0000:ffff2000       __guard_fids__             10000000     MSVCRT:std_type_info_static.obj
 0000:ffff2000       __guard_fids__             10000000     MSVCRT:throw_bad_alloc.obj
 0000:ffff2000       __guard_fids__             10000000     MSVCRT:throw_bad_alloc.obj
 0000:ffff2000       __guard_fids__             10000000     MSVCRT:throw_bad_alloc.obj
 0000:ffff2000       __guard_fids__             10000000     MSVCRT:throw_bad_alloc.obj
 0000:ffff2000       __guard_fids__             10000000     MSVCRT:throw_bad_alloc.obj
 0000:ffff2000       __guard_fids__             10000000     MSVCRT:throw_bad_alloc.obj
 0000:ffff2000       __guard_fids__             10000000     MSVCRT:throw_bad_alloc.obj
 0000:ffff2000       __guard_fids__             10000000     MSVCRT:throw_bad_alloc.obj
 0000:ffff2000       __guard_fids____scrt_set_unhandled_exception_filter 10000000     MSVCRT:utility_desktop.obj
 0000:ffff0000       .debug$S                   10000000     vcruntime:VCRUNTIME140.dll
 0000:ffff0000       .debug$S                   10000000     vcruntime:VCRUNTIME140.dll
 0000:ffff0000       .debug$S                   10000000     vcruntime:VCRUNTIME140.dll
 0000:ffff0000       .debug$S                   10000000     vcruntime:VCRUNTIME140.dll
 0000:ffff0000       .debug$S                   10000000     vcruntime:VCRUNTIME140.dll
 0000:ffff0000       .debug$S                   10000000     vcruntime:VCRUNTIME140.dll
 0000:ffff0000       .debug$S                   10000000     vcruntime:VCRUNTIME140.dll
 0000:ffff0000       .debug$S                   10000000     vcruntime:VCRUNTIME140.dll
 0000:ffff0000       .debug$S                   10000000     vcruntime:VCRUNTIME140.dll
 0000:ffff0000       .debug$S                   10000000     vcruntime:VCRUNTIME140.dll
 0000:ffff0000       .debug$S                   10000000     vcruntime:VCRUNTIME140.dll
 0000:ffff0000       .debug$S                   10000000     vcruntime:VCRUNTIME140.dll
 0000:ffff0000       .debug$S                   10000000     ucrt:api-ms-win-crt-heap-l1-1-0.dll
 0000:ffff0000       .debug$S                   10000000     ucrt:api-ms-win-crt-heap-l1-1-0.dll
 0000:ffff0000       .debug$S                   10000000     ucrt:api-ms-win-crt-heap-l1-1-0.dll
 0000:ffff0000       .debug$S                   10000000     ucrt:api-ms-win-crt-heap-l1-1-0.dll
 0000:ffff0000       .debug$S                   10000000     ucrt:api-ms-win-crt-runtime-l1-1-0.dll
 0000:ffff0000       .debug$S                   10000000     ucrt:api-ms-win-crt-runtime-l1-1-0.dll
 0000:ffff0000       .debug$S                   10000000     ucrt:api-ms-win-crt-runtime-l1-1-0.dll
 0000:ffff0000       .debug$S                   10000000     ucrt:api-ms-win-crt-runtime-l1-1-0.dll
 0000:ffff0000       .debug$S                   10000000     ucrt:api-ms-win-crt-runtime-l1-1-0.dll
 0000:ffff0000       .debug$S                   10000000     ucrt:api-ms-win-crt-runtime-l1-1-0.dll
 0000:ffff0000       .debug$S                   10000000     ucrt:api-ms-win-crt-runtime-l1-1-0.dll
 0000:ffff0000       .debug$S                   10000000     ucrt:api-ms-win-crt-runtime-l1-1-0.dll
 0000:ffff0000       .debug$S                   10000000     ucrt:api-ms-win-crt-runtime-l1-1-0.dll
 0000:ffff0000       .debug$S                   10000000     ucrt:api-ms-win-crt-runtime-l1-1-0.dll
 0000:ffff0000       .debug$S                   10000000     ucrt:api-ms-win-crt-runtime-l1-1-0.dll
 0000:ffff0000       .debug$S                   10000000     ucrt:api-ms-win-crt-runtime-l1-1-0.dll
 0000:ffff0000       .debug$S                   10000000     ucrt:api-ms-win-crt-runtime-l1-1-0.dll
 0000:ffff0000       .debug$S                   10000000     ucrt:api-ms-win-crt-runtime-l1-1-0.dll
 0000:ffff0000       .debug$S                   10000000     ucrt:api-ms-win-crt-stdio-l1-1-0.dll
 0000:ffff0000       .debug$S                   10000000     ucrt:api-ms-win-crt-stdio-l1-1-0.dll
 0000:ffff0000       .debug$S                   10000000     ucrt:api-ms-win-crt-stdio-l1-1-0.dll
 0000:ffff0000       .debug$S                   10000000     ucrt:api-ms-win-crt-string-l1-1-0.dll
 0000:ffff0000       .debug$S                   10000000     dbgeng:dbgeng.dll
 0000:ffff0000       .debug$S                   10000000     kernel32:KERNEL32.dll
 0000:ffff0000       .debug$S                   10000000     kernel32:KERNEL32.dll
 0000:ffff0000       .debug$S                   10000000     kernel32:KERNEL32.dll
 0000:ffff0000       .debug$S                   10000000     kernel32:KERNEL32.dll
 0000:ffff0000       .debug$S                   10000000     kernel32:KERNEL32.dll
 0000:ffff0000       .debug$S                   10000000     kernel32:KERNEL32.dll
 0000:ffff0000       .debug$S                   10000000     kernel32:KERNEL32.dll
 0000:ffff0000       .debug$S                   10000000     kernel32:KERNEL32.dll
 0000:ffff0000       .debug$S                   10000000     kernel32:KERNEL32.dll
 0000:ffff0000       .debug$S                   10000000     kernel32:KERNEL32.dll
 0000:ffff0000       .debug$S                   10000000     kernel32:KERNEL32.dll
 0000:ffff0000       .debug$S                   10000000     kernel32:KERNEL32.dll
 0000:ffff0000       .debug$S                   10000000     kernel32:KERNEL32.dll
 0000:ffff0000       .debug$S                   10000000     kernel32:KERNEL32.dll
 0000:ffff0000       .debug$S                   10000000     kernel32:KERNEL32.dll
 0000:ffff0000       .debug$S                   10000000     kernel32:KERNEL32.dll
 0000:ffff0000       .debug$S                   10000000     kernel32:KERNEL32.dll
 0000:ffff0000       .debug$S                   10000000     kernel32:KERNEL32.dll
 0001:00000e80       ?addLoadObjects@@YA_NPAUJNIEnv_@@PAV_jobject@@@Z 10001e80 f   sawindbg.obj
 0001:00001130       ?addThreads@@YA_NPAUJNIEnv_@@PAV_jobject@@@Z 10002130 f   sawindbg.obj
 0001:000016f0       ?attachToProcess@@YA_NPAUJNIEnv_@@PAV_jobject@@J@Z 100026f0 f   sawindbg.obj
 0001:00001820       ?getWindbgInterfaces@@YA_NPAUJNIEnv_@@PAV_jobject@@@Z 10002820 f   sawindbg.obj
 0001:00001b10       ?openDumpFile@@YA_NPAUJNIEnv_@@PAV_jobject@@PAV_jstring@@@Z 10002b10 f   sawindbg.obj
 0001:00001ca0       ?releaseWindbgInterfaces@@YA_NPAUJNIEnv_@@PAV_jobject@@@Z 10002ca0 f   sawindbg.obj
 0001:00001e40       ?setImageAndSymbolPath@@YA_NPAUJNIEnv_@@PAV_jobject@@@Z 10002e40 f   sawindbg.obj
 0001:00002000       ?throwNewDebuggerException@@YAXPAUJNIEnv_@@PBD@Z 10003000 f   sawindbg.obj
 0001:00003330       _event_to_env              10004330 f   sadis.obj
 0001:000033c0       _getLastErrorString        100043c0 f   sadis.obj
 0001:000034a0       _printf_to_env             100044a0 f   sadis.obj
 0001:000036b0       $$000000                   100046b0     MSVCRT:chkstk.obj
 0001:000036c4       cs10                       100046c4     MSVCRT:chkstk.obj
 0001:000036d2       cs20                       100046d2     MSVCRT:chkstk.obj
 0001:000036e5       ?dllmain_crt_dispatch@@YGHQAUHINSTANCE__@@KQAX@Z 100046e5 f   MSVCRT:dll_dllmain.obj
 0001:0000374c       ?dllmain_crt_process_attach@@YAHQAUHINSTANCE__@@QAX@Z 1000474c f   MSVCRT:dll_dllmain.obj
 0001:00003894       ?dllmain_crt_process_detach@@YAH_N@Z 10004894 f   MSVCRT:dll_dllmain.obj
 0001:00003970       ?dllmain_dispatch@@YAHQAUHINSTANCE__@@KQAX@Z 10004970 f   MSVCRT:dll_dllmain.obj
 0001:00003abd       ?dllmain_raw@@YGHQAUHINSTANCE__@@KQAX@Z 10004abd f   MSVCRT:dll_dllmain.obj
 0001:0000413e       ___get_entropy             1000513e f   MSVCRT:gs_support.obj
 0001:0000427d       ?find_pe_section@@YAPAU_IMAGE_SECTION_HEADER@@QAEI@Z 1000527d f   MSVCRT:utility.obj
 0001:000042d7       ?is_potentially_valid_image_base@@YA_NQAX@Z 100052d7 f   MSVCRT:utility.obj
 0001:000049d0       $$000000                   100059d0     MSVCRT:sehprolg4.obj
 0001:00004a30       $$000000                   10005a30     MSVCRT:sehprolg4.obj
 0001:00004b2d       ___castguard_check_failure_os_handled_wrapper 10005b2d f   MSVCRT:guard_support.obj
 0001:00004b89       ___castguard_check_failure_user_handled_wrapper 10005b89 f   MSVCRT:guard_support.obj
 0001:00004baf       ___castguard_compat_check  10005baf f   MSVCRT:guard_support.obj
 0001:00004d03       ___castguard_slow_path_compat_check 10005d03 f   MSVCRT:guard_support.obj
 0001:00006480       __ehhandler$??1?$AutoCOMPtr@UIDebugClient@@@@QAE@XZ 10007480 f   sawindbg.obj
 0001:000064b0       __ehhandler$??1?$AutoCOMPtr@UIDebugControl@@@@QAE@XZ 100074b0 f   sawindbg.obj
 0001:000064e0       __ehhandler$??1AutoJavaString@@QAE@XZ 100074e0 f   sawindbg.obj
 0001:00006510       __unwindfunclet$?addLoadObjects@@YA_NPAUJNIEnv_@@PAV_jobject@@@Z$0 10007510 f   sawindbg.obj
 0001:0000651d       __ehhandler$?addLoadObjects@@YA_NPAUJNIEnv_@@PAV_jobject@@@Z 1000751d f   sawindbg.obj
 0001:00006560       __unwindfunclet$?addThreads@@YA_NPAUJNIEnv_@@PAV_jobject@@@Z$0 10007560 f   sawindbg.obj
 0001:00006568       __unwindfunclet$?addThreads@@YA_NPAUJNIEnv_@@PAV_jobject@@@Z$1 10007568 f   sawindbg.obj
 0001:00006575       __ehhandler$?addThreads@@YA_NPAUJNIEnv_@@PAV_jobject@@@Z 10007575 f   sawindbg.obj
 0001:000065b0       __unwindfunclet$?openDumpFile@@YA_NPAUJNIEnv_@@PAV_jobject@@PAV_jstring@@@Z$0 100075b0 f   sawindbg.obj
 0001:000065bd       __ehhandler$?openDumpFile@@YA_NPAUJNIEnv_@@PAV_jobject@@PAV_jstring@@@Z 100075bd f   sawindbg.obj
 0001:000065f0       __unwindfunclet$?setImageAndSymbolPath@@YA_NPAUJNIEnv_@@PAV_jobject@@@Z$0 100075f0 f   sawindbg.obj
 0001:000065f8       __unwindfunclet$?setImageAndSymbolPath@@YA_NPAUJNIEnv_@@PAV_jobject@@@Z$1 100075f8 f   sawindbg.obj
 0001:00006605       __ehhandler$?setImageAndSymbolPath@@YA_NPAUJNIEnv_@@PAV_jobject@@@Z 10007605 f   sawindbg.obj
 0001:00006630       __ehhandler$_Java_sun_jvm_hotspot_debugger_windbg_WindbgDebuggerLocal_attach0__Ljava_lang_String_2Ljava_lang_String_2@16 10007630 f   sawindbg.obj
 0001:00006660       __ehhandler$_Java_sun_jvm_hotspot_debugger_windbg_WindbgDebuggerLocal_consoleExecuteCommand0@12 10007660 f   sawindbg.obj
 0001:00006690       __ehhandler$_Java_sun_jvm_hotspot_debugger_windbg_WindbgDebuggerLocal_lookupByName0@16 10007690 f   sawindbg.obj
 0002:0000111c       _GS_ExceptionPointers      1000a11c     MSVCRT:gs_report.obj
 0002:00002118       __ehfuncinfo$_Java_sun_jvm_hotspot_debugger_windbg_WindbgDebuggerLocal_attach0__Ljava_lang_String_2Ljava_lang_String_2@16 1000b118     sawindbg.obj
 0002:0000213c       __unwindtable$_Java_sun_jvm_hotspot_debugger_windbg_WindbgDebuggerLocal_attach0__Ljava_lang_String_2Ljava_lang_String_2@16 1000b13c     sawindbg.obj
 0002:00002174       __ehfuncinfo$_Java_sun_jvm_hotspot_debugger_windbg_WindbgDebuggerLocal_consoleExecuteCommand0@12 1000b174     sawindbg.obj
 0002:00002198       __unwindtable$_Java_sun_jvm_hotspot_debugger_windbg_WindbgDebuggerLocal_consoleExecuteCommand0@12 1000b198     sawindbg.obj
 0002:00002210       __unwindtable$_Java_sun_jvm_hotspot_debugger_windbg_WindbgDebuggerLocal_lookupByName0@16 1000b210     sawindbg.obj
 0002:00002220       __ehfuncinfo$_Java_sun_jvm_hotspot_debugger_windbg_WindbgDebuggerLocal_lookupByName0@16 1000b220     sawindbg.obj
 0002:0000224c       __ehfuncinfo$??1AutoJavaString@@QAE@XZ 1000b24c     sawindbg.obj
 0002:00002274       __ehfuncinfo$?setImageAndSymbolPath@@YA_NPAUJNIEnv_@@PAV_jobject@@@Z 1000b274     sawindbg.obj
 0002:00002298       __unwindtable$?setImageAndSymbolPath@@YA_NPAUJNIEnv_@@PAV_jobject@@@Z 1000b298     sawindbg.obj
 0002:000022dc       __ehfuncinfo$?openDumpFile@@YA_NPAUJNIEnv_@@PAV_jobject@@PAV_jstring@@@Z 1000b2dc     sawindbg.obj
 0002:00002300       __unwindtable$?openDumpFile@@YA_NPAUJNIEnv_@@PAV_jobject@@PAV_jstring@@@Z 1000b300     sawindbg.obj
 0002:00002344       __unwindtable$?addLoadObjects@@YA_NPAUJNIEnv_@@PAV_jobject@@@Z 1000b344     sawindbg.obj
 0002:0000234c       __ehfuncinfo$?addLoadObjects@@YA_NPAUJNIEnv_@@PAV_jobject@@@Z 1000b34c     sawindbg.obj
 0002:00002374       __unwindtable$?addThreads@@YA_NPAUJNIEnv_@@PAV_jobject@@@Z 1000b374     sawindbg.obj
 0002:00002384       __ehfuncinfo$?addThreads@@YA_NPAUJNIEnv_@@PAV_jobject@@@Z 1000b384     sawindbg.obj
 0002:000023b0       __ehfuncinfo$??1?$AutoCOMPtr@UIDebugClient@@@@QAE@XZ 1000b3b0     sawindbg.obj
 0002:000023d8       __ehfuncinfo$??1?$AutoCOMPtr@UIDebugControl@@@@QAE@XZ 1000b3d8     sawindbg.obj
 0002:00002400       __sehtable$?dllmain_crt_process_attach@@YAHQAUHINSTANCE__@@QAX@Z 1000b400     MSVCRT:dll_dllmain.obj
 0002:00002420       __sehtable$?dllmain_crt_process_detach@@YAH_N@Z 1000b420     MSVCRT:dll_dllmain.obj
 0002:00002450       __sehtable$?dllmain_dispatch@@YAHQAUHINSTANCE__@@KQAX@Z 1000b450     MSVCRT:dll_dllmain.obj
 0002:00002520       __sehtable$___scrt_is_nonwritable_in_current_image 1000b520     MSVCRT:utility.obj
 0002:000026b0       .edata                     1000b6b0     sawindbg.exp
 0002:000026d8       rgpv                       1000b6d8     sawindbg.exp
 0002:00002704       rgszName                   1000b704     sawindbg.exp
 0002:00002730       rgwOrd                     1000b730     sawindbg.exp
 0002:00002746       szName                     1000b746     sawindbg.exp
 0002:00002753       $N00001                    1000b753     sawindbg.exp
 0002:00002784       $N00002                    1000b784     sawindbg.exp
 0002:000027bc       $N00003                    1000b7bc     sawindbg.exp
 0002:00002804       $N00004                    1000b804     sawindbg.exp
 0002:00002871       $N00005                    1000b871     sawindbg.exp
 0002:000028c5       $N00006                    1000b8c5     sawindbg.exp
 0002:00002909       $N00007                    1000b909     sawindbg.exp
 0002:0000295c       $N00008                    1000b95c     sawindbg.exp
 0002:000029a0       $N00009                    1000b9a0     sawindbg.exp
 0002:000029ee       $N00010                    1000b9ee     sawindbg.exp
 0002:00002a39       $N00011                    1000ba39     sawindbg.exp
 0003:0000044c       ?imagePath_ID@@3PAU_jfieldID@@A 1000c44c     sawindbg.obj
 0003:00000450       ?symbolPath_ID@@3PAU_jfieldID@@A 1000c450     sawindbg.obj
 0003:00000454       ?ptrIDebugClient_ID@@3PAU_jfieldID@@A 1000c454     sawindbg.obj
 0003:00000458       ?ptrIDebugControl_ID@@3PAU_jfieldID@@A 1000c458     sawindbg.obj
 0003:0000045c       ?ptrIDebugDataSpaces_ID@@3PAU_jfieldID@@A 1000c45c     sawindbg.obj
 0003:00000460       ?ptrIDebugOutputCallbacks_ID@@3PAU_jfieldID@@A 1000c460     sawindbg.obj
 0003:00000464       ?ptrIDebugAdvanced_ID@@3PAU_jfieldID@@A 1000c464     sawindbg.obj
 0003:00000468       ?ptrIDebugSymbols_ID@@3PAU_jfieldID@@A 1000c468     sawindbg.obj
 0003:0000046c       ?ptrIDebugSystemObjects_ID@@3PAU_jfieldID@@A 1000c46c     sawindbg.obj
 0003:00000470       ?addLoadObject_ID@@3PAU_jmethodID@@A 1000c470     sawindbg.obj
 0003:00000474       ?addThread_ID@@3PAU_jmethodID@@A 1000c474     sawindbg.obj
 0003:00000478       ?createClosestSymbol_ID@@3PAU_jmethodID@@A 1000c478     sawindbg.obj
 0003:0000047c       ?setThreadIntegerRegisterSet_ID@@3PAU_jmethodID@@A 1000c47c     sawindbg.obj
 0003:0000048c       ?__proc_attached@@3HA      1000c48c     MSVCRT:dll_dllmain.obj
 0003:00000490       _GS_ExceptionRecord        1000c490     MSVCRT:gs_report.obj
 0003:000004e0       _GS_ContextRecord          1000c4e0     MSVCRT:gs_report.obj
 0003:00000874       ?is_initialized_as_dll@@3_NA 1000c874     MSVCRT:utility.obj
 0003:00000875       ?module_local_atexit_table_initialized@@3_NA 1000c875     MSVCRT:utility.obj
 0003:00000878       ?module_local_atexit_table@@3U_onexit_table_t@@A 1000c878     MSVCRT:utility.obj
 0003:00000884       ?module_local_at_quick_exit_table@@3U_onexit_table_t@@A 1000c884     MSVCRT:utility.obj
 0004:000004f6       .idata$6                   1000d4f6     dbgeng:dbgeng.dll
 0004:00000690       .idata$6                   1000d690     kernel32:KERNEL32.dll
 0004:0000079a       .idata$6                   1000d79a     vcruntime:VCRUNTIME140.dll
 0004:0000092c       .idata$6                   1000d92c     ucrt:api-ms-win-crt-stdio-l1-1-0.dll
 0004:0000094c       .idata$6                   1000d94c     ucrt:api-ms-win-crt-heap-l1-1-0.dll
 0004:0000096c       .idata$6                   1000d96c     ucrt:api-ms-win-crt-runtime-l1-1-0.dll
 0004:0000098e       .idata$6                   1000d98e     ucrt:api-ms-win-crt-string-l1-1-0.dll
